:0A000000803102288801883124288D
:10001E00640080010131890B1028003421009913EE
:10002E0019179916191699118B0191019201200039
:10003E009101920122008C01383021008C002300A6
:10004E008C0122008E01303021008E0023008E01A3
:10005E002100950124008E150E168E168C150C1689
:10006E008C1621009513200098019C012500930108
:10007E009A012400950182302200970090302100D1
:10008E009E007D309D000C3026009A0025009E13A8
:10009E001E170F3028009600260098000430280006
:1000AE0097008B13230091013F309505151413080B
:1000BE002000D9000130230091003F309505151422
:1000CE0013082000DC000230230091003F3095051C
:1000DE00151413082000DF000330230091003F3079
:1000EE009505151413082000DD000430230091003F
:1000FE003F309505151413082000DE00053023004F
:10010E0091003F309505151413082000E1000630CC
:10011E00230091003F309505151413082000D800D8
:10012E000730230091003F30950515141308200069
:10013E00E3000830230091003F3095051514130895
:10014E002000E2000930230091003F309505151480
:10015E0013082000DA000B30912780311030F200A6
:10016E002730F3000525803170082000D400710877
:10017E00D500890D893B8909D600D7000C3091270F
:10018E008031E830F2000330F300052580316F270F
:10019E0080310D30912780316430F200F301052556
:1001AE0080316F2780310E30912780310A30F20076
:1001BE00F301052580316F270F30230091003F306A
:1001CE009505151413082000D40701300318D50720
:1001DE000318D6070318D7076308DB008831C2203F
:1001EE008031DA2380318A258B31FA238031003039
:1001FE008831E42080310030AB260030893159211E
:10020E00803120005C08A00059089F3109278031F9
:10021E00A42780310030F9268C1021308E31D4265F
:10022E00803120006208B73E8E31D42680312030D6
:10023E008E31D426803120005A08031928290D301A
:10024E0029290C308E31D42680318C14E027803150
:10025E00470820005F06F0395F062100C700200026
:10026E009A278031031D40160B302000BB001C3036
:10027E00BA006330B900B90B4229BA0B4229BB0B45
:10028E00422964000E248031332680310230200052
:10029E00BB000330BA00BA30B900B90B5429BA0BFF
:1002AE005429BB0B54298A258B31FA238031953181
:1002BE005525803151088831E42080319F31D22775
:1002CE00803120004C0E0F398931592180312000A8
:1002DE008C1A8229BB2180312000DD080030031DDD
:1002EE007F299E313826803120008C1A82297B2965
:1002FE009D31D025803120000C1A9629BB218031EA
:10030E002000DD080130031D93299E3138268031EF
:10031E0020000C1A96298F299D31D025803120007E
:10032E008C199D29BB218031E12180318E1AA9299A
:10033E00BB2180312000DF0310305F020318DF0184
:10034E004627803120000E1AB829BB2180312000AB
:10035E00DF0A10305F02031CB6290F30DF0046277C
:10036E008031BB2180314D2920008C1A0C1EC429EE
:10037E008C198E1EC4290E1AC6296308DB0050087C
:10038E004F060319CF294F08D0005B08031DDB036E
:10039E00DB08031DD52926009801D8295808260008
:1003AE00980020006308633A031D08000F302600F2
:1003BE0098000800DA238C31B5248031F03021000A
:1003CE00C705F023803120008C19FA290230B800BD
:1003DE000330B700BA30B600B60BF329B70BF329CA
:1003EE00B80BF329EA298A25803150084F060319E4
:1003FE00052A4F08D0008C31B524803120008C1A8C
:10040E00212AE40B0D2AE401E40ACE030B304E023E
:10041E000318CE018C31B524803103302000B80092
:10042E008830B7005630B600B60B1B2AB70B1B2A06
:10043E00B80B1B2A20000C1A422AE40A063064026A
:10044E00031C2C2A0530E400CE0A0B304E02031C8E
:10045E00322A0A30CE008C31B52480310330200090
:10046E00B8008830B7005630B600B60B3C2AB70B32
:10047E003C2AB80B3C2A200064084E07CB008E1A8B
:10048E000E1E5D2BC42B8E1A4E2ADD01DD0A0E1EAA
:10049E00DD0123009518502A0330910020005D08DD
:1004AE009731CD278031031C8B2B8B178B2B8E1AFC
:1004BE00622ADE01DE0A0E1EDE0123009518642A72
:1004CE000430910020005E08572A8E1EE1010E1A9C
:1004DE00722AE101E10A23009518722A0530910073
:1004EE0020006108572A8E1A832AC7031830470244
:1004FE00031C832A1730C7000E1A8A2AC70A18301F
:10050E0047020318C701292580318B2B8E1A962A94
:10051E00C9033C304902031C962A3B30C9000E1A0F
:10052E009D2AC90A3C3049020318C901452580316C
:10053E008B2B8E1AA92ACF033C304F02031CA92AFB
:10054E003B30CF000E1AB02ACF0A3C304F020318B0
:10055E00CF01612580318B2B8E1AB92AC60BB92A91
:10056E000730C6000E1AC22AC60A08304602031CFD
:10057E00C22AC601C60A7D2580318B2B8E1ACB2A44
:10058E00C50BCB2A1F30C5000E1AD42AC50A20303F
:10059E004502031CD42AC501C50A8831A320803127
:1005AE008B2B8E1ADE2ACA0BDE2A0C30CA000E1ACC
:1005BE00E72ACA0A0D304A02031CE72ACA01CA0AF0
:1005CE008831842080318B2B8E1AF42AD20364302A
:1005DE005202031CF42A6330D2000E1AFB2AD20AEE
:1005EE00643052020318D2018831652080318B2B82
:1005FE008E1A082BD80310305802031C082B0F300C
:10060E00D8000E1A0F2BD80A103058020318D80132
:10061E00230095180F2B0630910020005808572AFA
:10062E008E1A202BE30364306302031C202B6330ED
:10063E00E3000E1A272BE30A643063020318E3016A
:10064E0023009518272B0730910020006308572AA6
:10065E008E1A362BE203153062020318E2010E1ACF
:10066E003F2BE20A15306202031C3F2B1430E200CE
:10067E00230095183F2B0830910020006208572A5E
:10068E008E1EDA010E1A4D2BDA01DA0A23009518A6
:10069E004D2B0930910020005A08572A8E1E592BD7
:1006AE000E1A8B2B8931E22180318B2B4B08013AAC
:1006BE0003194A2A033A03195E2A013A03196C2ACE
:1006CE00073A03197A2A013A03198D2A033A0319B4
:1006DE00A02A013A0319B32A0F3A0319C52A013A7F
:1006EE000319D82A033A0319EB2A013A0319FF2AF0
:1006FE00073A0319172B013A03192F2B033A031943
:10070E00472B013A0319552B200058082600980054
:10071E0022008C1020005A080319972B0D30982BAD
:10072E000C308E31D426803121308E31D42680315A
:10073E0020006208B73E8E31D426803120308E31B3
:10074E00D42680318C148C31B524803103302000B6
:10075E00B8008830B7005630B600B60BB42BB70BC6
:10076E00B42BB80BB42B20009A278031031D4016F2
:10077E00F023803120006308DB008C19FA29DA237C
:10078E0080313326803120008C1908000230B800E9
:10079E000330B700BA30B600B60BD32BB70BD32B42
:1007AE00B80BD32BCA2BF10100308931D621803101
:1007BE00F301F40101307402F830031973020318C7
:1007CE00080000308E31D4268031F30A0319F40A62
:1007DE00E12B7F2480312030612480314008612458
:1007EE008031410861248031420861248031430800
:1007FE0061248031440861248031450861248031B0
:10080E00460861248031470861248031242D200060
:10081E005908F000F101E830F2000330F30005252D
:10082E0080317108F7007008F6005C08F000F101E5
:10083E000A30F200F301052580317008F6077108C1
:10084E00F73D2030F607D730F73D77082100CC0072
:10085E007608CD007F24803120306124803140081D
:10086E006124803141086124803142086124803145
:10087E004308612480314408612480314508612495
:10088E008031460861248031470861248031480850
:10089E00612480314908612480314A086124803105
:1008AE004B08612480314C08612480314D0861244D
:1008BE008031242DF1000830F200F2080319792C52
:1008CE00F2037108F000720A6D2CF036890B6C2C55
:1008DE00701C742C22000E15762C22000E111D2574
:1008EE008031642C21000E151D2521000E110800EB
:1008FE0022000E158E151A2580310E111A258E1115
:10090E000800FB007608F10002308931D6218031D3
:10091E00FC01FD0100307D020C3003197C0203182E
:10092E00AB2C7B08F000F1010C30F200F301052531
:10093E0080310130F700903082278E31D4268031FD
:10094E00FC0A0319FD0A912C00308E31D426803119
:10095E0000308E31D42680317608F1000330893193
:10096E00D6218031FC01FD0100307D020C300319CF
:10097E007C020318D52C7B08F000F1010C30F2003C
:10098E00F301052580317930F700903082278E31C2
:10099E00D4268031FC0A0319FD0ABB2C00308E319F
:1009AE00D426803100308E31D42680317608F10085
:1009BE0004308931D6218031FC01FD0100307D02E9
:1009CE000C3003197C020318FF2C7B08F000F10198
:1009DE000C30F200F30105258031F130F700903034
:1009EE0082278E31D4268031FC0A0319FD0AE52CAC
:1009FE0000308E31D42600308E31D42EF401F50124
:100A0E00701C0D2D7208F4077308F53DF235F30DC9
:100A1E00F136F00C71087004031D072D7508F100F6
:100A2E007408F00008000000000008001A2580314C
:100A3E0022008E151A258E11080022008E151A25F9
:100A4E000E1508007F248031D030612480310230B1
:100A5E0061240A30F000200047088F31382780319A
:100A6E00F9000A30F50047088F3120278031890EB2
:100A7E00F0397907FA0061248031242D7F248031EA
:100A8E00D03061248031013061240A30F000200022
:100A9E0049088F3138278031F9000A30F5004908AE
:100AAE008F3120278031890EF0397907FA006124C1
:100ABE008031242D7F248031D0306124803100306C
:100ACE0061240A30F00020004F088F313827803122
:100ADE00F9000A30F5004F088F3120278031890E3A
:100AEE00F0397907FA0061248031242D7F2480317A
:100AFE00D0306124803103306124803120004608DB
:100B0E0061248031242D7F248031D03061248031C6
:100B1E00003061248031242580317F248031D13012
:100B2E0061248031082680312000CF0024268031B8
:100B3E00082680312000C900242680310826803105
:100B4E002000C70024268031082680312000C600F0
:100B5E0024268031082680312000C50024268031CD
:100B6E00082680312000CA002426803108268031D4
:100B7E002000D2006C278031242580310F302000D8
:100B8E004F05F3000A30F0004F0E0F392726803143
:100B9E007307CF000F304905F3000A30F000490EFD
:100BAE000F39272680317307C9000F304705F30030
:100BBE000A30F000470E0F39272680317307C70021
:100BCE000F304505F3000A30F000450E0F39272689
:100BDE0080317307C5000F304A05F3000A30F0006C
:100BEE004A0E0F39272680317307CA000F3052057F
:100BFE00F3000A30F000520E0F3927267307D20089
:100C0E000800F1010830F20021000E15F208031958
:100C1E00202EF20320000E1D1D2E0130F000720A50
:100C2E00192EF035890B182E7008F1041D25803110
:100C3E000D2E21000E117108080022000E111D2D1F
:100C4E00F200F10170087218F107F035F236F20871
:100C5E00031D292E710808008A258B31FA23803155
:100C6E00200051088831E42080310030AB2600305E
:100C7E0089315921803120005C08A00059089F312C
:100C8E0009278031A42720005E088831402080315A
:100C9E000030F92680312000AB0120005F082B02C6
:100CAE000318752EAB0A2B08AB268031210047089E
:100CBE0020002B06F0392B062100C700F0238031CF
:100CCE0002302000A8000330A700BA30A600A60B01
:100CDE006E2EA70B6E2EA80B6E2E542E5230A90020
:100CEE00AA019F31F527803105257108A7005C0800
:100CFE007002A600031CA703303EF8002A30273DE1
:100D0E00F9009E31C92680317608A9027708AA3BE0
:100D1E00AB0120002B08A600A7012A082702031DFD
:100D2E009A2E2908260203180800AB0A2B08F9266A
:100D3E0080311A302000A700F830A600A60BA52E91
:100D4E00A70BA52E6400902EF7003030F100013075
:100D5E008931D62180310A30282780310A30770236
:100D6E00031CC82E0130DC2600308E31D426803193
:100D7E000A30F00077088F3138278031DC26803139
:100D8E00D92E77080319D42E0A30F00077088F3148
:100D9E0038278031DC268031D72E0B302827803142
:100DAE002D30282700308E31D42EF300F40104307C
:100DBE00740203180800730809070907D43EF100EE
:100DCE0092300318890AF2007408710784007208C1
:100DDE000318720A8500000809078E31D426803167
:100DEE00F40ADE2EF40053307402031C002F52302E
:100DFE00F400F10105308931D62180317408523C5E
:100E0E00F300FC308E31D4268031F4037408FF3A9F
:100E1E000319172FB430092F84308E31D426803128
:100E2E00F3037308FF3A031D132FFC308E31D426C3
:100E3E0080315330F10005308931D621FC308E31AE
:100E4E00D42EF500F60105307602031808000530A1
:100E5E00F00075082726693EF30091300318890AC1
:100E6E00F40076087307840074080318740A85006A
:100E7E00000809078E31D4268031F60A2A2F210068
:100E8E00470820005F06F0395F062100C700F023F7
:100E9E00803120005F08AB2680310230FA0003302B
:100EAE00F900BA30F800F80B5A2FF90B5A2FFA0B3B
:100EBE005A2F23009518602F0230910020005F08F2
:100ECE009731CD2703188B17080022000E151D2D04
:100EDE0070082000B9007108BA000030BA1BFF304C
:100EEE00BB00BC003908D4073A08D53D3B08D63DB7
:100EFE003C08D73D0800F80070087707F900710824
:100F0E00783DFA0079087C0784007A087D3D8500DB
:100F1E0000080800230091003F30950515141308B2
:100F2E00F000F10108005E082100C012031DC0167A
:100F3E00200061082100401208003930F100033012
:100F4E008931D6218031F301F401003074021B3057
:100F5E00031973020318C22F7308683E840092307F
:100F6E000318013E850000088E31D4268031F30A25
:100F7E000319F40AAC2F3930F10004308931D6212F
:100F8E008031F301F401003074021B300319730237
:100F9E00031808007308833E840092300318013E44
:100FAE00850000088E31D4268031F30A0319F40A25
:100FBE00CA2F2100C01740174016C0164010411509
:100FCE0041144308F3390838C300FC390238C30012
:100FDE00C6170F30C60447083F398038C7000F3098
:100FEE00C7044A0883394038CA00CA14CB144B14BC
:020FFE000800E9
:101048003D30840000308500173080310F20883112
:10105800A0308400003085002E3080310F20083009
:10106800E0000130E1000A30E2001430E300013012
:10107800E400200080311528F3003930F1000230F7
:10108800D6218831F401F501003075021B300319AF
:101098007402031808007308031957287408B93E26
:1010A800840092305B2874089E3E840092300318B6
:1010B800013E85000008D4268831F40A0319F50A90
:1010C800482884317F248831D030843161248831A4
:1010D80006308431612488310A30F000200052083B
:1010E80038278831F9000A30F50052082027890E80
:1010F800F0397907FA008431612488318531242D4B
:1011080084317F248831D03084316124883105309E
:101118008431612488310A30F00020004A083827D9
:101128008831F9000A30F5004A082027890EF0397D
:101138007907FA008431612488318531242D84317E
:101148007F248831D030843161248831043084315F
:10115800612488310A30F00020004508382788319A
:10116800F9000A30F50045082027890EF03979077B
:10117800FA008431612488318531242D22000C1431
:101188008C102130D42688311330D426883104308D
:10119800D4268831C230D42688312030D4268831EC
:1011A8000930D42688310830D42688310C30D4262A
:1011B80088318030D42688314030D4268C140800F9
:1011C800FC003030F1000030D621883164307C02D8
:1011D800031CF4286430F5007C0820278831F528A2
:1011E8000A30502788310030D42688310A307C02F2
:1011F8000A30031C0729F5006430F0007C08382702
:10120800883120278831502788310030D42688310A
:101218006430F0007C0838278831FA000A30F00082
:101228007A0838278831502788310030D426883109
:101238000030D42688310C30B62688310030D426C8
:1012480088310030D42688310030D42688311C30CB
:10125800D42688317F30D426883164307C02031C40
:1012680037296330FC000A30F5007C0820278831D4
:10127800FB00093CF900F9037908FF3A03194A29E8
:101288004130D42688313F29D4268831FB037B0896
:10129800FF3A7F30031D4829D42688315330F100A6
:1012A8000030D62188317F30D42EF4004030F10050
:1012B8000130D6218831F3011430730203186929EB
:1012C8000030D4268831F30A60294030F10001301B
:1012D800D62188310230D42688310430D42688318A
:1012E8000830D4268831FE30D42688310830D426F8
:1012F80088310430D42688310230D42688314530EC
:10130800F1000130D62188317408031991298430FD
:10131800D42688310230D426883102307402031C66
:101328009B29C030D42688310030D4268831033038
:101338007402031CA529E030D42688310030D42655
:10134800883104307402031CAF29F030D426883168
:101358000030D426883105307402031CB929F830CE
:10136800D42688310030D426883106307402031C14
:10137800C329FC30D42688310030D4268831073080
:101388007402031CCD29FE30D42688310030D426BF
:10139800883108307402031C0800FF30D4268831D5
:1013A8000030D42EF20022008C107208403ED42661
:1013B80088317108803ED4268C1408002100470823
:1013C80020005F06F0395F062100C7008331F02353
:1013D80088318331DA23883109302000D300BD01F8
:1013E800BE01BF01C0019731532788312000C20ACE
:1013F800073042020318C20120008C1E052A8E1AEB
:10140800122AC40354304402031C0C2A5330C4006B
:10141800440897317A2788312000CD0A0C1E162AF5
:101428000E1A212AC40A543044020318C40144087D
:1014380097317A2788312000CD0A8C1D0800CD0A03
:1014480053304D02031C2A2AAE30CD075308031926
:10145800322A48089531B2258831A42AF101023090
:10146800D62188312000C208031D402A6730F700C2
:101478009330F800FF2688312000420B492A4A3071
:10148800F7009330F800FF26883120004208023A1E
:10149800031D542ABB30F7009330F800FF2688312B
:1014A80020004208033A031D5F2AD730F700933023
:1014B800F800FF26883120004208043A031D6A2AF2
:1014C8008330F7009330F800FF2688312000420867
:1014D800053A031D752A9F30F7009330F800FF2660
:1014E800883120004208063A031DA42A4030F7003C
:1014F8009430F800FF2688310930B626883100304C
:10150800D42688310930B62688310030D42688316F
:101518000930B62688310030D42688310930B626FD
:1015280088310030D42688310930B6268831003019
:10153800D42688310230F7009430F800FF2688312D
:10154800200040085702031DB32A3F085602031D16
:10155800B32A3E085502031DB32A3D085402031856
:10156800BD2A4008D7003F08D6003E08D5003D08F0
:10157800D4001830F1000030D6212000A301A201C8
:101588002730A1001030A0005708A7005608A60071
:101598005508A5005408A40097311427883120085D
:1015A800502788310030D42688312000A301A201B9
:1015B8000330A100E830A0005708F7005608F600ED
:1015C8005508F5005408F400F301F2012730F10042
:1015D8001030F000C42388319B27973114278831B5
:1015E8002008502788310030D42664302000A0001D
:1015F800A101A201A3019731DD278831C4238831D5
:101608006B278831C42388319B2797311427883169
:101618002008502788310030D4260A302000A00046
:10162800A101A201A3019731DD278831C4238831A4
:101638006B278831C423883173087A278831C423FB
:1016480088319B2797311427883120085027883103
:101658000030D42620009731DD278831C423883113
:101668006B278831C423883173087A278831C423CB
:101678008831AF278831C4238831700850278831D2
:101688000030D42688313B30F1000030D6212000CC
:10169800A301A2012730A1001030A0004008A70034
:1016A8003F08A6003E08A5003D08A400973114276E
:1016B80088312008502788310030D426883120000E
:1016C800A301A2010330A100E830A000A4278831BB
:1016D8002730F1001030F000C42388319B27973160
:1016E800142788312008502788310030D4268831C3
:1016F800643087278831C42388316B278831C42315
:1017080088319B2797311427883120085027883142
:101718000030D42688310A3087278831C42388319D
:101728006B278831C423883173087A278831C4230A
:1017380088319B2797311427883120085027883112
:101748000030D42688312000A42788310330F100E6
:10175800E830F000C42388316B278831C4238831EE
:1017680073087A278831C4238831AF278831C42386
:1017780088317008502788310030D4268831002AF3
:1017880073087204710470040319F12BF801F80A44
:10179800F31BD32BF035F10DF20DF30DCB2B7308A2
:1017A8007702031DE12B72087602031DE12B7108F5
:1017B8007502031DE12B70087402031CEB2B7008E3
:1017C800F4027108F53B7208F63B7308F73BF336F1
:1017D800F20CF10CF00CF80BD32B7708F300760819
:1017E800F2007508F1007408F0000800F1010030FB
:1017F800D62188310A30F500200047082027883193
:10180800B62688310030D42688310A30F00020000E
:10181800470838278831B62688310030D4268831E1
:101828000030D42688313630D42688313630D42654
:1018380088310030D42688310030D42688310A30E7
:10184800F5002000490820278831B6268831003065
:10185800D42688310A30F00020004908382788311A
:10186800B62688310030D42688310030D426883115
:101878003630D42688313630D42688310030D42604
:1018880088310030D42688310A30F50020004F080E
:1018980020278831B62688310030D42688310A308E
:1018A800F00020004F0838278831B6268831F1012A
:1018B8000130D62188312000F62787312827883142
:1018C8000030D4268831EB27873128278831F90161
:1018D8000F3079020318752C0030D4268831F90AA4
:1018E8006C2C0E30F1000130D62188310A30F50019
:1018F8002000450820278831003A03198B2C0A302C
:10190800F50045082027873128278831902C113089
:10191800F1000130D62188310030D42688310A30D0
:10192800F0002000450838278731282788311C30E7
:10193800F1000130D62188312000DF2787312827A0
:1019480088310030D4268831D2278731282788313A
:101958000030D4268831C5278731282788310030C0
:10196800D42EF1010030D6218831F330F7009330BE
:10197800F800FF268831FA01FA0A632E5D08031978
:10198800C92CBD30F7009430CC2CB930F700943016
:10199800F800FF2688315C30F7009430F800FF2605
:1019A8008831632E5E080319DD2CB030F7009430BF
:1019B800E02CA430F7009430F800FF2688318030FE
:1019C800F7009430F800FF268831632E6108031968
:1019D800F12CB530F7009430F42CAB30F70094308C
:1019E800F800FF2688318930F7009430F800FF2688
:1019F8008831632E0A30F500470820278831B6263B
:101A080088310030D42688310A30F0002000470899
:101A180038278831B62688315330F7009430F800DB
:101A2800FF268831632E0A30F500490820278831BF
:101A3800B62688310030D42688310A30F0002000DC
:101A4800490838278831B62688316E30F700943037
:101A5800F800FF268831632E0A30F5004F0820274A
:101A68008831B62688310030D42688310A30F00013
:101A780020004F0838278831B62688314A30F700C9
:101A88009430F800FF268831632EF6278831B62671
:101A980088310030D4268831EB278831B626883142
:101AA8009230F7009430F800FF268831632E0A3010
:101AB800F500450820278831B62688310030D4261D
:101AC80088310A30F0002000450838278831B626CA
:101AD80088316530F7009430F800FF268831632E8E
:101AE800DF278831B62688310030D4268831D227BE
:101AF8008831B62688310030D4268831C527883108
:101B0800B62688310030D42688317730F7009430F3
:101B1800F800FF268831632E0230B626883100305F
:101B2800D42688310030B62688310030D426883152
:101B38000A30F5002000520820278831B62688315F
:101B48000030D42688310A30F000200052083827A7
:101B58008831B62688319B30F7009430F800FF268C
:101B68008831632E0A30F500580820278831B626B8
:101B780088310030D42688310A30F0002000580817
:101B880038278831B62688313430F7009430F80089
:101B9800FF268831632E0A30F50063082027883134
:101BA800B62688310030D42688310A30F00020006B
:101BB800630838278831B62688311030F70094300A
:101BC800F800FF268831632E0A30F50062082027C6
:101BD8008831B62688310030D42688310A30F000A2
:101BE8002000620838278831B62688311C30F70073
:101BF8009430F800FF268831632E2D30B6268831C0
:101C08000030D426883120005A08B626883128307A
:101C1800F7009430F800FF268831632E2E30B62660
:101C280088310030D42688312E30B62688310030ED
:101C3800D42688312E30B62688310030D426883113
:101C48004030D42688310030D42688312F30B6264B
:101C580088310030D42688310D30B62688310030DE
:101C6800D42688310F30B62688310030D426883102
:101C78001730B62688310030D42688313030B62661
:101C880088310030D42688311F30B626883100309C
:101C9800D42688314030D42688310030D426883183
:101CA8003130B62688310030D42688313230B62615
:101CB80088312D30B62688312D30B6268831063049
:101CC8007A02F1010318A42E7A08D62188312D3022
:101CD800B62688310030D426883120004E087A078D
:101CE800F900FA0A013A0319C22C033A0319D62C4F
:101CF800013A0319EA2C073A0319FE2C013A031991
:101D0800172D033A0319302D013A0319492D0F3ABB
:101D180003195B2D013A0319742D033A0319902D09
:101D2800013A0319B62D073A0319CF2D013A0319C1
:101D3800E82D033A0319012E013A0319122E632ED6
:101D480020006408D62188317F30D42688313E307F
:101D5800D42688311C30D42688310830D4268831DE
:101D68000030D42EF500F60105307602031808007D
:101D78000530F0007508863127268831693EF30062
:101D880091300318890AF4007608730784007408F0
:101D98000318740A85000008D4268831F60AB82E7C
:101DA800F00022000C11F01B0C150E100E140C1173
:101DB800701B0C150E100E140C11F01A0C150E10C9
:101DC8000E140C11701A0C150E100E140C11F019BB
:101DD8000C150E100E140C1170190C150E100E1493
:101DE8000C11F0180C150E100E140C1170180C159F
:101DF8000E100E1408007708840078088500000883
:101E0800003803190800770884007808850000085E
:101E1800203A0319162F77088400780885000008EF
:101E28004D3E172F2D30B6268831F70A0319F80AC8
:101E38000030D4268831FF2EF600F8017508031902
:101E4800362FF701F70AF51B2B2FF535262FF83516
:101E580075087602031C332F7508F6027814F536D8
:101E6800F70B2B2F78080800F2000830F300F40174
:101E78007208F1000730F136890B3F2F7435710471
:101E8800F400F23570087402031C4C2F7008F40239
:101E9800F30B3C2F74080800F300F40104307402BB
:101EA80003180800730809070907D43EF1009230A7
:101EB8000318890AF200740871078400720803186D
:101EC800720A85000008D4268831F40A522F730854
:101ED800F7007208F6007108F5007008F400F301C5
:101EE800F2010330F100E830F0000800F700720852
:101EF800F6007108F5007008F4006430F000F10194
:101F0800F201F30108002000A000A101A201A30131
:101F18004008F7003F08F6003E08F5003D08F400C9
:101F2800F301F2010330F100E830F0000800730813
:101F3800A7007208A6007108A5007008A400080090
:101F48004008F7003F08F6003E08F5003D08F40099
:101F5800F301F20108007308B5007208B4007108B3
:101F6800B3007008B2000A30F000F101F201F30189
:101F78003508F7003408F6003308F5003208F40095
:101F8800080020004A0809074A07023E84009330E7
:101F98000318013E850000084D3E080020004A084D
:101FA80009074A07013E840093300318013E850063
:101FB80000084D3E08004A0809074A07003E840009
:101FC80093300318013E850000084D3E08002000AC
:101FD8004635293E840093300318013E85000008E9
:101FE8004D3E08004635283E840093300318013ED4
:101FF800850000084D3E08000034F034F0343034D9
:102008003034303430343034303430343034F034E8
:10201800F034003400340034C034C034F034F034C8
:102028000034003400340034003430343034303478
:102038003034303430343034303430343034F034B8
:10204800F0343034303430343034303430343034A8
:10205800303430343034F034F034F034F034003488
:102068000034003400340034003400340034F034D8
:10207800F034F034F03430343034303430343034F8
:1020880030343034303430343034F034F0343034A8
:102098003034303430343034303430343034303418
:1020A8003034303430343034303430343034303408
:1020B800303430343034F034F034F034F0343034F8
:1020C8003034303430343034303430343034F03428
:1020D800F034F034F0343034303430343034303498
:1020E800303430343034F034F034FF34FF340034DA
:1020F8000034003400340034003400340034FF3439
:10210800FF3400340034003400340034FF34FF342A
:1021180000340034003400340034F034F034303407
:1021280030343034303430343034303430343F3478
:102138003F34003400340034003430343034303428
:10214800303430343034FF34FF343F343F343034AB
:102158003034303430343034303430343034FF3488
:10216800FF343F343F34303430343034303430345A
:10217800303430343034F034F034FF34FF34303419
:102188003034303430343034303430343034F03467
:10219800F034003400340034003400348034C03467
:1021A800E034703438341F340F34FF34FF343034A3
:1021B8003034303430343034303430343034FF3428
:1021C800FF343F343F3430343034303430343034FA
:1021D800303430343034FF34FF343F343F3430341B
:1021E80030343034303430343034303430343F34B8
:1021F8003F34003400340034303430343F343F341A
:10220800303430340034003400343F343F34303418
:102218003034303430343034303430343034303496
:102228003034303430343034303430343034303486
:102238003034303430343F343F34003400340034E8
:1022480000340034003400340034003400343F34A7
:102258003F34303430343034303430343034303447
:102268003034303430343F343F343F343F3430340A
:1022780030343034303430343034303430343F3427
:102288003F34003400340034003400343F343F34E9
:10229800003400340034003400343F343F343034E8
:1022A80030343034303430343034303430343F34F7
:1022B8003F343034303430343034303430343034E7
:1022C8003034303430343F343F347F344134413457
:1022D80041347F34003442347F344034003479341C
:1022E8004934493449344F34413441344934493408
:1022F8007F340F340834083408347F344F34493479
:102308004934493479347F34493449344934793447
:10231800013401347134093407347F344934493481
:1023280049347F344F344934493449347F341C3478
:102338001C3422347F3400342234143408341434E6
:102348002234263416340834343432347E3411348A
:10235800113411347E347F344934493449343134AA
:102368007F3449344934493436347F3401340134B4
:102378000134033440347E34413441347F347F3473
:102388004934493449344134673418347F34183473
:102398006734223441344934493436347F34203464
:1023A800103408347F347F342034113408347F34B7
:1023B8007F34083408341434633440347E340134B0
:1023C80001347F347F340234043402347F347F3460
:1023D8000834083408347F343E34413441344134BD
:1023E8003E347F340134013401347F347F3409347E
:1023F8000934093406343E344134413441342234FA
:10240800013401347F34013401340734483448340A
:1024180048343F341E3421347F3421341E3463342D
:1024280014340834143463347F34403440347F34F3
:10243800403407340834083408347F347F34403457
:102448007E3440347F347F3440347E3440347F34AB
:1024580001347F344834483430347F344834483485
:1024680030347F3400347F344834483430342234B4
:102478004134493449343E347F3408343E3441349D
:102488003E3446342934193409347F340034003456
:102498000034003400343F344034383440343F345E
:1024A8007F344034403440346034003441347F3425
:1024B800413400347F3409341934293446343F34E4
:1024C8004034403440343F34FC34F8347034E03421
:1024D800C034E0347034F834FC3400340034FC3454
:1024E800FC340C340C340C340C341C341C34803460
:1024F80080340034003400348034803400343F3475
:102508003F34003400340134003400343F343F3465
:10251800003400343F343F34003400340034003495
:10252800003400343F343F343034303430343F34B6
:102538007F34603470348834883488340034083404
:10254800F83408340034F834A83488340034F834C3
:102558002834283410340034F834A834883400344B
:1025680070348834883488347034F8341034203423
:10257800403420341034F8340034703488348834CB
:102588008834883470340034F834203420342034CB
:10259800F83400347034883488348834883470349B
:1025A8007F34413441347F34003442347F34403402
:1025B8007934493449344F344134493449347F34C7
:1025C8000F34083408347F344F344934493479346B
:1025D8007F34493449347934013471340934073447
:1025E8007F34493449347F344F34493449347F3453
:1025F8000034003400340034D534D534D534DF34D5
:10260800CD34C234D434C534C234CC34C034D034DC
:10261800C034CF34D034CC34C034DF34C834DE34A2
:10262800CD34C834DE34CB34C034C234C334D134AE
:10263800C534CD34CE34CA34D234CD34CE34DF347C
:10264800C434C534CA340034D534D534CF34CD3449
:10265800C234D234D134D034D734D234CF34D23453
:10266800D134C134C234D13400340E341F343F3431
:102678007E34FC347E343F341F340E34013403344A
:1026880007340F341F343F347F34FF34D034C03420
:10269800C734CE34CC34CD34C8342034CF34C034ED
:1026A800CB34DC34D634DB34C8342034CF34CE34A5
:1026B800CF34D034CE34C134D334C9342034C534C3
:1026C800D934C534003420342034CD34C034CC342B
:1026D8002034D234C034CA34C034DF3420342034F7
:1026E8002034C834C334D034C0342034CD34C53455
:1026F8002034CD34D334C634CD34C0340034D1344E
:10270800CB34C534C434D334DE34D934C034DF34A4
:102718002034C834C334D034C03420342034C134D5
:10272800D334C434C534D2342034CB34C534C33460
:10273800D734C5340034203420342034CC34CE345B
:10274800DF342034CC34C034CC34C034203420348A
:1027580020342034C834C334D034C034C534D234DF
:102768002034CB34D334D734D834C5340034CD34C2
:10277800C5342034D134D234C034D034C034C53414
:10278800D834DC34D134DF3420342034CC34CE3463
:10279800C634C534D834DC342034CB34D334D734BD
:1027A800D834C53400342034CE34D734C534CD348D
:1027B800DC342034D134C834CB34DC34CD34CE349A
:1027C8002034C434C034C234C834D834DC3420345F
:1027D800CA34CD34CE34CF34CA34C834003420346B
:1027E800CD34C034D134D234D034CE34C934CA34E0
:1027F800C83420342034203420340034C834203401
:10280800C134D334C434C534D2342034CC34D33472
:10281800CB34DC34D23400342034D134C234C5341F
:10282800D2342034D134C534CA342034203400346E
:102838002034CA34CE34CD34D234D034C034D13438
:10284800D2342034203400342034C834CD34C23457
:10285800C534D034D134C834DF3420342034003483
:102868002034DF34D034CA34CE34D134D234DC34DA
:102878002034203420340034CD34C034C134C5343D
:10288800D034C534D834DC34203400342034D13446
:10289800C534CA34D334CD34C4342034003420345D
:1028A800D734C034D134CE34C23420342034003448
:1028B8002034CF34CE34C834D134CA342034203410
:1028C80000342034D734C834D134CB34CE34203417
:1028D800203400342034CC34C834CD34D334D2340A
:1028E8002034203400342034CC34C534D134DF349F
:1028F800D6342034203400342034C734C234D3349E
:10290800CA3420342034203400342034C134C03454
:10291800D134DB3420342034203400342034C4341F
:10292800C534CD34DC342034203420340034203411
:10293800C334CE34C434203420342034203400341A
:10294800D134D234C534D034C534CE340034CE3446
:10295800D234CA34CB340034CC34CE34CD34CE3433
:102968000034C234CA34CB340034C034C234D23414
:0A2978000034D034D334D7340034D7
:102AAA0021009D149D18572D1C08F300F401F40011
:102ABA00F3011B08F304023074025830031973023D
:102ACA0003187B2D5830F0000230F10073087002B1
:102ADA00F3007408713BF400003074026530031986
:102AEA007302031C7D2D6430F3007C2DF301F40185
:102AFA0020005108F000F10174087106031D872DAA
:102B0A007308700603190800C10A2030410203182D
:102B1A00C1014108A03E8600870173088100F201C5
:102B2A00F301F401203072020318A52D7208A03EA9
:102B3A00860087010108F3070318F40AF20A972DA1
:102B4A007408F1007308F0000530F136F00C890BB7
:102B5A00AA2D70082000D1000800B100F100600819
:102B6A00AD00AD36AD36AD362D088931D621953159
:102B7A00F5278E31D4269531F5278E31D426953115
:102B8A002000C30A02304302031CCD2DC301E00A10
:102B9A00B0014B304402031CD52D4408B53EB000A9
:102BAA00480830020318EE2D44084802031C0E2E72
:102BBA004408073EAD00003003180130AE00803AE9
:102BCA00AF0080302F02031DEC2D48082D02031C94
:102BDA000E2E2000BD0A0319BE0A0319BF0A0319E3
:102BEA00C00A00304002031D042E01303F02031DBB
:102BFA00042E86303E02031D042EA0303D02031C23
:102C0A00182EC0010130BF008630BE009F30BD00C3
:102C1A00182E303020006002031C182ED3035327CD
:102C2A0095314B269531303020006002031C080094
:102C3A000830E000303060020318452E3108F100F8
:102C4A006008AD00AD36AD36AD362D088931D621D6
:102C5A009531F527FF3A8E31D4269531F527FF3A7B
:102C6A008E31D42695310D302000AE00FB30AD00F8
:102C7A00AD0B3D2EAE0B3D2E422E2000E00A1F2E3C
:102C8A000830E0004D08C80044087A2F2000A3014C
:102C9A00A2012730A1001030A0005708A70056084B
:102CAA00A6005508A5005408A40014279531200849
:102CBA00AC00230095185E2E0B30910020002C08E2
:102CCA00CD2703188B172000A301A2010330A1000E
:102CDA00E830A0005708F7005608F6005508F50036
:102CEA005408F400F301F2012730F1001030F0002B
:102CFA008B31C42395318F319B2795311427953118
:102D0A002008AC0023009518872E0C309100200073
:102D1A002C08CD27953103188B1764302000A000AA
:102D2A00A101A201A301DD278B31C42395318F3183
:102D3A006B2795318B31C42395318F319B27953180
:102D4A00142795312008AC0023009518A92E0D30C0
:102D5A00910020002C08CD27953103188B170A30D3
:102D6A002000A000A101A201A301DD278B31C42309
:102D7A0095318F316B2795318B31C4239531730887
:102D8A008F317A2795318B31C42395318F319B2727
:102D9A009531142795312008AC0023009518D22EBE
:102DAA000E30910020002C08CD27953103188B177F
:102DBA002000DD278B31C42395318F316B27953164
:102DCA008B31C423953173088F317A2795318B3132
:102DDA00C42395317308AB007208AA007108A900D0
:102DEA007008A8000A30F000F101F201F3012B0883
:102DFA00F7002A08F6002908F5002808F4008B31A4
:102E0A00C42395317008AC0023009518092F0F30A0
:102E1A00910020002C08CD2703188B170800F90110
:102E2A00FA01FB01FC0123082204210420040319EE
:102E3A004A2FFD01FD0AA31B272FA035A10DA20DC4
:102E4A00A30D1F2FF935FA0DFB0DFC0D23082702E0
:102E5A00031D392F22082602031D392F21082502B6
:102E6A00031D392F20082402031C442F2008A40222
:102E7A002108A53B2208A63B2308A73B7914A336C1
:102E8A00A20CA10CA00CFD0B272F7C08A3007B0829
:102E9A00A2007A08A1007908A0000800F101003018
:102EAA008931D6219531F5010930750203186A2F47
:102EBA007508393E840093300318013E85000008E6
:102ECA008E31D4269531F50A592F00308E31D42609
:102EDA00953100308E31D4269531200053088F3138
:102EEA005027953100308E31D42EF600F5014B3043
:102EFA007602031C832F7608B53EF500F1010530F2
:102F0A008931D6219531F701543077020318080028
:102F1A0075087702031CC52F770876060319C52F93
:102F2A007608013EEC2795310319C52F7608023E33
:102F3A00EC2795310319C52F7608033EEC27953106
:102F4A000319C52F7608043EEC2795310319C52FBE
:102F5A007608053EEC2795310319C52F7608063EFB
:102F6A00EC2795310319C52F7608073EEC279531D2
:102F7A000319C52F7608083EEC279531031DC72F84
:102F8A00C030C82F00308E31D4269531F70A892FE8
:102F9A00230093003F30950503108B1B03148B13FA
:102FAA00151555309600AA3096009514151108008B
:102FBA005708F7005608F6005508F5005408F400BB
:102FCA00F301F2010330F100E830F0000800F300E9
:102FDA00003003180130F4007708730674040800FF
:102FEA00200060080739423E840093300318013EEE
:062FFA008500000808003C
:103BA000A80028080319E82D0A30DC075B305C0206
:103BB000031CDC2DDC01D90A59086C3A031DFC2DCD
:103BC0005C080319FC2D5730D9005A30DC00FC2D5D
:103BD000F630DC075B305C02031CF12D5A30DC0050
:103BE000D9035908573A031DFC2D5A305C020318BB
:103BF000FC2D6C30D900DC0184310E249D31200075
:103C00005C08A000590809279D3152302000A90006
:103C1000AA01F527853105259D317108A7005C08AB
:103C20007002A600031CA703303EF8002A30273D8F
:103C3000F900C9267608A9027708AA3B2908863127
:103C4000F9269D3123009518222E91012000590854
:103C50009731CD279D3103188B1795182D2E0130E4
:103C6000910020005C089731CD2703188B170800BE
:103C7000AA00CC0120004C18B32E2A080319542E98
:103C80000A30DC075B305C02031C482EDC01D90AD9
:103C900059086C3A031D682E5C080319682E5730CA
:103CA000D9005A30DC00682EF630DC075B305C024D
:103CB000031C5D2E5A30DC00D9035908573A031D06
:103CC000682E5A305C020318682E6C30D900DC0173
:103CD00084310E249D3120005C08A000590809277A
:103CE0009D3168302000A700E430A600A60B762E98
:103CF000A70B762E6400D22720004C0E0F39893195
:103D000059219D3120008C1A892E2A0B892EAA0157
:103D1000CC010C1A912EAA08031D912EAA01AA0A01
:103D2000CC018C198E1E08000E1E08005230A8000F
:103D3000A901F527853105259D317108A7005C088B
:103D40007002A600031CA703303EF8002A30273D6E
:103D5000F900C9267608A8027708A93B2808863109
:103D6000F9269D313A2E23009518B32E910120009B
:103D700059089731CD279D3103188B179518BE2E02
:103D80000130910020005C089731CD2703188B1774
:103D90000800FB01F71FD32EF609F709F60A0319ED
:103DA000F70AFB01FB0AF91FDC2EF809F909F80AEA
:103DB0000319F90A0130FB06FC01FD0177087604BE
:103DC0000319FC2EFA01FA0AF71BE92EF635F70D56
:103DD000E32EFC35FD0D77087902031DF12E7608E0
:103DE0007802031CF82E7608F8027708F93B7C1459
:103DF000F736F60CFA0BE92E7B080319042FFC09A1
:103E0000FD09FC0A0319FD0A7D08F7007C08F6008D
:103E10000800A5006430F50025088F3120279D316A
:103E2000A1006430F00025088F3138279D31A300B0
:103E30000A30F50023088F3120279D31A30064301C
:103E4000F00025088F3138279D31A4000A30F0009A
:103E500024088F3138279D31A4000A30F50020084E
:103E60008F3120279D31A20021080319392F0130FD
:103E70003A2F003057270830F600200023088431FD
:103E800088249D311630F6002000240884318824CF
:103E90009D3130308E31D4269D3130308E31D42654
:103EA0009D312830F600200022088431882CF30050
:103EB000F10102308931D6219D31F401F501003044
:103EC00075020630031974020318792F7308031959
:103ED000712F1030740784009030753D8500000804
:103EE000722F00308E31D4269D31F40A0319F50A61
:103EF0005F2F00308E31D4269D3100308E31D42694
:103F00009D31F10103308931D6219D31F401F50154
:103F1000003075020630031974020318A22F7308CB
:103F200003199A2F8830740784009030753D8500FE
:103F300000089B2F00308E31D4269D31F40A0319DE
:103F4000F50A882F00308E31D4269D3100308E3115
:103F5000D4269D31F10104308931D6219D31F401FF
:103F6000F501003075020630031974020318CB2FD7
:103F700073080319C32F0030740784009130753D16
:103F800085000008C42F00308E31D4269D31F40AFC
:103F90000319F50AB12F00308E31D4269D3100303F
:103FA0008E31D42E84317F249D312130843161249F
:103FB0009D31863108269D31F300F401F400F301B0
:103FC000863124269D31863108269D31F30703185A
:103FD000F40A863124269D31863108269D31200041
:103FE000CC0087316C278531242D1930F600F7017C
:103FF0005908F000F1019C30F200FF30F300080096
:020000040001F9
:04000E0024EFFF1CC0
:10E0000065000A0003000000000001000F0014007A
:10E010000A000000FF0000000000000000000000F7
:00000001FF
